:020000020000FC
:100000000FC075C08BC08DC098C098C088C088C014
:0400100097C095C040
:10002000F89400E810E006BD16BD0EE90DBF06E02D
:1000300008BB0DE107BBB0E0A0E6D0E0C0EA00E0FD
:100040000D93BD17E9F7AC17D9F701E005BF00E044
:1000500004BF00E005BD00E002BF00E00FBD00E00E
:1000600003BF00E006BF00E009BD00E008BD00E2FC
:1000700007B900E006B900E003B900E004BB00E8FE
:1000800008B90EE1102F01BD11BD00E40BBF00E067
:1000900005BB02E009BF00E60ABF0EE008BF00E0B2
:1000A000002E18E300E4312E202E90E07894A895DD
:1000B00090FFFDCF9E7F20EC32E140E455E6132D0A
:1000C000022D41D008F412C038E320E4021B130BC8
:1000D000201B310B209530950894201D301D22BF28
:1000E000532E02E008BFC29801E003BFE0CFFFB685
:1000F000B1990AC070E073BF302C02BE926072E00A
:1001000078BF71E073BF08C070E073BF78940000DF
:10011000F89422B69D7F9160FFBE189518951895AA
:100120001895FFB63394539419F4C29A60E063BFF4
:10013000FFBE189518951895189518951895189547
:100140001895189518956F937F93712F602F621BE8
:10015000730B28F0712F602F461B570B00F07F9117
:100160006F9108951F932F932BE117E71A95F1F7DD
:0E0170002A95D9F70A95C1F72F911F9108958E
:00000001FF
